:1000000099C5C3C5D1C575C8B0C5D4C8AEC5AEC540
:10001000ACC5ABC577C7A9C5A8C5A7C5A6C500010E
:10002000904C9132009880810000904C9132009564
:1000300080810094904C913200948081009A904885
:100040009132009580810000904C91320093808124
:100050000094904F00998001BE90379143009980A1
:10006000810092002500250025002600260026009C
:100070002600269048913700250074808101299040
:1000800043913400948081012F90409130009380FF
:1000900081012E904591350092000380810022005D
:1000A00025002500250001904791370024002500F8
:1000B000260026808100000099904691360092002B
:1000C0000380810000904591350022002500250025
:1000D0002500018081002400250026002690439100
:1000E00034006780810064904C913C006380810003
:1000F00064904F9140006080810064905191410074
:100100009980810095904D913E00938081000090F0
:100110004F914000948081009A904C913C009580D2
:1001200081009490489139009480810000904A9118
:100130003B00998081000090479137009200038036
:10014000810022002500250026002600260026002A
:1001500026904891370026007480810129904391B0
:100160003400948081012F90409130009380810170
:100170002E904591350092000380810022002500D9
:100180002500250001904791370024002500260016
:1001900026808100000099904691360092000380ED
:1001A00081000090459135002200250025002500A2
:1001B0000180810024002500260026904391340010
:1001C0006780810064904C913C0063808100649062
:1001D0004F9140006080810064905191410099806E
:1001E000810095904D913E009380810000904F9149
:1001F0004000948081009A904C913C009580810051
:100200009490489139009480810000904A913B007D
:10021000998081000090479137009200038081000F
:100220002200250025002500250025002600269017
:100230003000998000920003904F00220025002595
:10024000002600018000009037914E002400260017
:1002500026002681800000904D002600748000005A
:10026000904B0095800000903C0093800000904CE3
:100270000094800000903500998000009044009523
:1002800080000090450093800000903C91480094CD
:1002900080810000903C0099800000904500920011
:1002A000038000009035914800220025002500259C
:1002B000000181800000904A0024002500260026CD
:1002C00080000090300099800095904F009380004E
:1002D000009034914E009480810000904D009980F0
:1002E0000000904B00958000009037009380000044
:1002F000904C913C00948081009A9054009580002D
:1003000094905400948000009054009980009200D2
:1003100003903700220025002500250001800024DD
:10032000002500260026903000998000920003905E
:100330004F00220025002500260001800000903794
:10034000914E002400260026002681800000904D5A
:1003500000260074800000904B0095800000903CC7
:100360000093800000904C0094800000903500992C
:10037000800000904400958000009045009380002C
:1003800000903C9148009480810000903C0099804E
:1003900000009045009200038000009035914800D5
:1003A00022002500250025000181800000904A00E0
:1003B000240025002600268000009030009980004F
:1003C00095904B913800938081012E904A913A008C
:1003D00095808101289048913C009980810092008D
:1003E0002500250025002600019037002400260066
:1003F000260026800000903700260074800095902B
:100400003000938000949030009980009200039017
:100410004F002200250025002600018000009037B3
:10042000914E002400260026002681800000904D79
:1004300000260074800000904B0095913C80009451
:10044000810000904C00948000009035009980005D
:10045000009044009580000090450093800000903B
:100460003C9148009480810000903C0099800000FD
:1004700090450092000380000090359148002200D2
:100480002500250025000181800000904A002400FD
:10049000250026002680000090300099800095906D
:1004A0004F00938000009034914E009480810000B2
:1004B000904D0099800000904B009580000090378F
:1004C0000093800000904C913C00948081009A90B1
:1004D0005400958000949054009480000090540043
:1004E0009980009200039037002200250025002506
:1004F000000180002400250026002690300099800D
:1005000000920003904F00220025002500260001E4
:100510008000009037914E0024002600260026819E
:10052000800000904D00260074800000904B0095E4
:10053000800000903C0093800000904C009480006C
:100540000090350099800000904400958000009054
:10055000450093800000903C914800948081000009
:10056000903C0099800000904500920003800000BC
:10057000903591480022002500250025000181804A
:100580000000904A002400250026002680000090EC
:10059000300099800095904B913800938081012E16
:1005A000904A913A0095808101289048913C0099A9
:1005B000808100920025002500250026000190374B
:1005C0000024002600260026800000903700260028
:1005D00074800095903000938000949048912C0096
:1005E0009980810000904800958000949033914854
:1005F00000948081009A9048009580000090389186
:100600004A0093808100949037914C00998081003A
:10061000009048009580009490309145009480812E
:10062000000090430099800095902B0093800094E7
:100630009048912C0099808100009048009580009E
:10064000949033914800948081009A90480095805E
:1006500000009038914A009380810000904C0094F3
:10066000800000903700998001299030009480012B
:100670002F902B00938000949048912C00998081BA
:100680000000904800958000949033914800948039
:1006900081009A90480095913880904A009481801A
:1006A00000949037914C009980810000904800950B
:1006B0008000949030914500948081000090430028
:1006C000998000920003902B00220025002500262F
:1006D0000001800024002600260026904C91320064
:1006E00026007480810000904C913200958081003A
:1006F00094904C913200948081009A9048913200FD
:100700009580810000904C913200938081009490FC
:100710004F00998001BE903700998000920025001B
:100720002500250026002600260026004D904C912D
:1007300030009980810000904800958000949036A8
:10074000914300948081000090370099800095903B
:1007500044913C00938081009490459135009980AC
:1007600081904D006C002500038000009035002230
:100770000025002500250001800000904D00240088
:100780002600260025800000903C9145009980813C
:100790000000903C006C00250003800000903500B4
:1007A00022002500250025000180002400260026C7
:1007B00000259047913200678000328100319051CE
:1007C00000638000649051003091350030800063F8
:1007D0008100009051913700678000328100319094
:1007E0004F0063800000903B0063914D003080001B
:1007F000308100649037914C0099808100009048CE
:100800000095800000903700938000009045009490
:10081000800000903C9143009980810000903C0052
:100820006C00250003800000903700220025002680
:10083000002600018000250026004D904C913000DC
:1008400099808100009048009580009490369143F3
:100850000094808100009037009980009590449129
:100860003C009380810094904591350099808100EF
:1008700000904D006C0025000380000090350022A0
:100880000025002500250001800000904D00240077
:100890002600260025800000903C9145009980812B
:1008A0000000903C006C00250003800000903500A3
:1008B00022002500250025000180002400260026B6
:1008C000002590479137009980810000904D009558
:1008D0008000949037914D00948081000090379172
:1008E0004D0067808100649039914C0063808100E5
:1008F00064903B914A006080810064903C91480084
:10090000998081000090400095800000903700930E
:10091000800000904000948000009030913C00994D
:100920008081006CF0650D0000310E0000090F00A1
:1009300000EE0F0000E0100000E1110000F21200D4
:1009400000121400004315000087160000DE170097
:100950000049190000CA1A0000621C0000121E00A3
:1009600000DC1F0000C1210000C3230000E32500BC
:100970000024280000872A00000E2D0000BC2F0054
:10098000009332000095350000C4380000243C007C
:1009900000B83F00008243000086470000C64B00BD
:1009A00000485000000E5500001D5A0000785F00FE
:1009B0000026650000296B0000897100004978005D
:1009C00000707F0000048700000B8F00008D9700EF
:1009D0000090A000001CAA000039B40000F1BE0085
:1009E000004BCA000053D6000011E3000092F00053
:1009F00000E0FE0000080E0100161E0100192F0184
:100A0000001F4101003854010073680100E27D01BC
:100A10000097940100A6AC010023C6010024E10167
:100A200000C0FD0100101C02002D3C0200335E02DC
:100A3000003F8202006FA80200E5D00200C3FB0263
:100A4000002E2903004B590300468C030048C203C3
:100A50000080FB0300203804005A78040066BC04C0
:100A6000007E040500DF500500CBA1050087F705D7
:100A7000005B52060097B206008B180700908407AF
:100A80000000F707003F700800B4F00800CC7809B8
:100A900000FB080A00BEA10A0096430B000DEF0BF5
:100AA00000B7A40C002E650D0017310E001F090FB2
:100AB0000001EE0F007FE0100067E1110097F112D6
:100AC00000F61114007B4315002B8716001ADE1761
:100AD000006D4919005BCA1A002D621C003F121EEE
:100AE0000002DC1F00FDC02100CFC223002FE32540
:100AF00000ED232800F7862A00560E2D0034BC2F67
:100B000000DB923200B79435005AC438007E243C92
:100B10000004B83F000102000004000102040810B4
:100B20002002020202020200000000360000000063
:100B30000038000011241FBECFE5D2E0DEBFCDBFDC
:100B400010E0A0E6B0E0EAEAF4E102C005900D9200
:100B5000A236B107D9F720E0A2E6B0E001C01D92AD
:100B6000A63AB207E1F799D49EC44ACA1F920F92DF
:100B70000FB60F9211248F9381E0809368008F91BC
:100B80000F900FBE0F901F9018951F920F920FB6E7
:100B90000F9211248F9381E0809366008F910F90C4
:100BA0000FBE0F901F9018951F920F920FB60F92C5
:100BB00011248F939F93809167008F5F80936700CC
:100BC0009091670080916000981730F01092670054
:100BD00098B380E1892788BB9F918F910F900FBEBA
:100BE0000F901F90189514BE81B5886181BD11BC0E
:100BF0000895CF93DF93F894F6DF80E48BBFD1E0C4
:100C0000D5BF88E187BBC4E0C8BB82E00BD480932A
:100C1000660080916600882331F083E08093600055
:100C2000D09369000FC081E870D3909365008093E2
:100C300064008536910524F082E08093600002C054
:100C4000C09360001092660080916900882361F172
:100C500081E85BD3909365008093640025E044E0D5
:100C600063E08AE690E058D08AE690E08BD06EE1AF
:100C700070E08AE690E030D1C8E080918700882358
:100C800089F081E842D390936300809362002091C1
:100C900064003091650020523340821793076CF74F
:100CA000C1BDEBCF8FE081BD88E088B993E094BBF4
:100CB0009AE090BD90E69BBF85BB7894DF91CF9181
:100CC000089580916800882349F0459B02C060E048
:100CD00001C061E083E05BD3109268008091660000
:100CE0008823C9F06EE170E080E090E0D4D2B29940
:100CF0000DC081E80AD39093650080936400853627
:100D0000910514F082E003C084E001C083E0809389
:100D10006000109266000895CF93DF93C62FD0E055
:100D2000D0939B00C0939A00A42FB0E0B093990099
:100D3000A0939800822F90E0909397008093960064
:100D4000E0E9F0E0D183C083B383A28395838483F9
:100D500081E090E0FC0102C0EE0FFF1F4A95E2F730
:100D6000AF01FC0102C0EE0FFF1F2A95E2F79F01C1
:100D7000240F01C0880F6A95EAF7820F87BBDF91C5
:100D8000CF91089582E08ABD83BF82E389BD80B799
:100D9000806880BF80B7826080BF80B7846080BF7A
:100DA00080B7816080BF80E48DBD10928700109273
:100DB0008F0010928E0010928D0010928C0080E5B2
:100DC00089BF78940895833060F590E06C3708F01F
:100DD0006BE7E62FF0E0EE0FFF1FEE0FFF1FEB5D5E
:100DE000F64F45915591659174919C01220F331FE7
:100DF000220F331FF901E159FF4F40835183628372
:100E00007383F901E558FF4F40E050E060E470E083
:100E10004083518362837383FC01E459FF4F21E0D7
:100E200020830895E0918800F0918900BF016F5FF1
:100E30007F4F7093890060938800849187FD10C074
:100E40003296F0938900E0938800FB01649170E092
:100E50006F5F7F4F782B70938F0060938E000895A3
:100E6000982F907F8F70903839F4E82FF0E0E45994
:100E7000FF4F108218BAD6CF903949F43296F093CA
:100E80008900E0938800FB0164919DDFCBCF903E09
:100E900049F480918A0090918B009093890080930F
:100EA0008800C0CF903F09F0BDCF1092870010920C
:100EB0006C0018BA10926D0018BA10926E0018BA31
:100EC0000895ECE6F0E0108218BA118218BA128286
:100ED00018BA109287000895CF93DF93EB01209109
:100EE00087002111EEDFD0938B00C0938A00D0934E
:100EF0008900C093880096DF81E080938700DF91AE
:100F0000CF9108951F920F920FB60F9211242F9335
:100F10004F935F936F937F938F939F93AF93BF9301
:100F200080916C00882309F444C040916F00509177
:100F30007000609171007091720080917B009091BF
:100F40007C00A0917D00B0917E00841B950BA60BC8
:100F5000B70B80937B0090937C00A0937D00B093AF
:100F60007E0080917B0090917C00A0917D00B091EB
:100F70007E00B7FF1EC028B381E090E000909A0089
:100F800002C0880F991F0A94E2F7822788BB8091DC
:100F90007B0090917C00A0917D00B0917E00A05CD0
:100FA000BF4F80937B0090937C00A0937D00B09313
:100FB0007E0080916D00882309F444C04091730045
:100FC00050917400609175007091760080917F005F
:100FD00090918000A0918100B0918200841B950BBC
:100FE000A60BB70B80937F0090938000A0938100A5
:100FF000B093820080917F0090918000A091810049
:10100000B0918200B7FF1EC028B381E090E000904D
:10101000980002C0880F991F0A94E2F7822788BBC4
:1010200080917F0090918000A0918100B09182001A
:10103000A05CBF4F80937F0090938000A0938100BD
:10104000B093820080916E00882309F444C04091DF
:101050007700509178006091790070917A008091CA
:10106000830090918400A0918500B0918600841B3C
:10107000950BA60BB70B8093830090938400A093ED
:101080008500B09386008091830090918400A091A8
:101090008500B0918600B7FF1EC028B381E090E0C4
:1010A0000090960002C0880F991F0A94E2F78227E9
:1010B00088BB8091830090918400A0918500B091BD
:1010C0008600A05CBF4F8093830090938400A09320
:1010D0008500B0938600BF91AF919F918F917F91D2
:1010E0006F915F914F912F910F900FBE0F901F90B6
:1010F00018951F920F920FB60F9211242F933F93C2
:101100004F935F936F937F938F939F93AF93BF930F
:10111000EF93FF9380916B00811124C08091870031
:10112000882389F080918E0090918F00892B59F04F
:1011300080918E0090918F00019790938F00809303
:101140008E00892B31F180918C0090918D00892B3C
:1011500049F080918C0090918D00019790938D00C3
:1011600080938C0090916B0081E0892780936B00C5
:10117000FF91EF91BF91AF919F918F917F916F916F
:101180005F914F913F912F910F900FBE0F901F9045
:10119000189548DED8CF80B7807F80BF80B7806841
:1011A00080BF8CB580648CBD8FEF8DBD80B78760AC
:1011B00080BF08951F920F920FB60F9211242F93A4
:1011C0003F938F939F93AF93BF9380919D00909196
:1011D0009E00A0919F00B091A00030919C0026E05D
:1011E000230F2D3730F029E8230F0396A11DB11DE1
:1011F00003C00296A11DB11D20939C0080939D0009
:1012000090939E00A0939F00B093A0008091A100B6
:101210009091A200A091A300B091A4000196A11DFD
:10122000B11D8093A1009093A200A093A300B0935E
:10123000A400BF91AF919F918F913F912F910F90FB
:101240000FBE0F901F9018953FB7F8948091A100A2
:101250009091A200A091A300B091A40022B708B67B
:1012600001FE05C02F3F19F00196A11DB11D3FBF22
:10127000BA2FA92F982F8827820F911DA11DB11D6C
:10128000BC01CD0143E0660F771F881F991F4A9567
:10129000D1F708950895CF92DF92EF92FF92CF9306
:1012A000DF936B017C01D0DFEB01C114D104E104B9
:1012B000F10479F0EFDFC8DF6C1B7D0B683E7340F3
:1012C000A0F381E0C81AD108E108F108C851DC4F49
:1012D000F2CFDF91CF91FF90EF90DF90CF90089504
:1012E0008AB582608ABD8AB581608ABD83B7887FEE
:1012F000836083BF789489B7826089BF4CDF86B1F1
:101300008877866886B9379A08958F709091A5007E
:101310009295990F990F907C892B87B987B19091FD
:10132000A50092FB222720F930E094E0220F331F22
:101330009A95E1F7282B27B9369A3699FECF84B1D2
:1013400025B190E0922B0895813031F48AB58F77E2
:101350008ABD8AB58F7B07C0823039F48AB58F7D0C
:101360008ABD8AB58F7E8ABD0895833039F480B7EF
:101370008F7D80BF80B78F7E80BF0895843031F429
:101380008CB58F7D8CBD8CB58F7E8CBD08950F93F1
:101390001F93CF93DF931F92CDB7DEB787FF11C0A6
:1013A0008F7741F0813041F0823041F0833041F05D
:1013B0008FEF07C085E005C082E003C084E001C074
:1013C00083E0282F30E0F901EB5EF44F8491F901BE
:1013D000E55EF44F1491F901EF5DF44F04910023A1
:1013E000D9F0882319F06983AFDF6981E02FF0E03D
:1013F000EE0FFF1FE35DF44FA591B4918FB761111C
:1014000006C0F8949C91E12FE095E92303C0F8947D
:10141000EC91E12BEC938FBF0F90DF91CF911F9157
:101420000F910895CF93DF9387FF11C08F7741F01D
:10143000813041F0823041F0833041F08FEF07C0BE
:1014400085E005C082E003C084E001C083E0282F6E
:1014500030E0F901EB5EF44F8491F901E55EF44F61
:10146000D491F901EF5DF44FC491CC2389F081113F
:101470006BDFEC2FF0E0EE0FFF1FE95DF44FA5915D
:10148000B491EC91ED2381E090E021F480E002C082
:1014900080E090E0DF91CF91089581B781BF20DF98
:0A14A000A8DB0FDCFECFF894FFCFAD
:0214AA0002003E
:00000001FF
